S00F0000526563697665722E7372656345
S11300000C942A000C9447000C9447000C9447006D
S11300100C9447000C9447000C9447000C94470040
S11300200C9447000C94C9000C9447000C944700AE
S11300300C9447000C9447000C9447000C94470020
S11300400C9447000C9447000C9447000C94470010
S11300500C94470011241FBECFE5D4E0DEBFCDBF12
S113006010E0A0E6B0E0E0EAF6E002C005900D92F0
S1130070A236B107D9F710E0A2E6B0E001C01D92A4
S1130080A636B107E1F70E9461010C944E030C946B
S1130090000080916000909161008630910511F11B
S11300A086E090E090936100809360008AEC90E099
S11300B090936300809362008FEF96E1A1E18150F9
S11300C09040A040E1F700C000001092630010923D
S11300D062008FEF96E1A1E181509040A040E1F7EA
S11300E000C0000008950895CF930E9427020E9443
S11300F034028823E1F70E943902882321F08A30F0
S113010011F0803FE1F50E9434028823E1F70E9458
S11301103902C82F0E9434028823E1F7C13079F5EF
S11301200E943902843051F0853018F4813039F559
S113013016C0853051F0873011F50EC082E090E092
S113014090936100809360000AC083E090E09093F4
S113015061008093600003C00E94490010C00E94A7
S11301603E028FE39CE90197F1F700C00000409143
S113017060005091610081E06AE00E94BB02CF916F
S1130180089585E083BF88E582BF1CBE81E089BFF6
S113019008951F920F920FB60F9211242F933F933D
S11301A08F939F9388E582BF809160009091610056
S11301B082309105D9F48091640090916500823376
S11301C0910554F480916400909165000196909398
S11301D06500809364000AC0B89AB09B02C0C098BE
S11301E001C0C09A10926500109264008091600072
S11301F09091610083309105D9F4809164009091CD
S113020065008530910554F48091640090916500F7
S1130210019690936500809364000AC0B89AB09BDD
S113022002C0C09801C0C09A109265001092640088
S1130230809160009091610086309105D9F480919D
S11302406400909165001816190654F080916400BA
S113025090916500019690936500809364000AC0B4
S1130260B89AB09B02C0C09801C0C09A10926500B1
S113027010926400B99AC19A8FEA94E00197F1F759
S113028000C0000080916200909163001816190666
S113029074F480E090E025E12A95F1F700000196DE
S11302A0209162003091630082179307A4F3C198F0
S11302B09F918F913F912F910F900FBE0F901F90A0
S11302C018950E94930180E296E00E94DB0181E090
S11302D060E047E00E94BD0180E895E20E94EB01E6
S11302E080E066E00E9412020E94C10078940E949D
S11302F07400FDCF949840E120E030E0992314F499
S1130300969A01C09698220F331F83992160959A7B
S1130310880F991F00C000009598415079F7949A6E
S1130320822F932F089581B3806781BB949A8FEFB6
S113033090E7A2E081509040A040E1F700C00000A7
S113034080EE90EC0E947A0187ED90E80E947A0199
S11303508BEA92EC0E947A0181E89AEC0E947A017D
S113036080E090EE0E947A0180E098EC0E947A018D
S113037087EF94EC0E947A01089590E0880F991F0A
S113038082959295907F9827807F9827907050E06F
S113039047705070842B952B946970E06370707073
S11303A0660F771F660F771F660F771F862B972BB5
S11303B00E947A0108958036910538F02FE0803448
S11303C0920728F08FE39FE002C080E690E0906AF5
S11303D00E947A01089522E08739920710F125E1FD
S11303E08831920780F49C0140E050E060E678EAAE
S11303F080E090E00E943303C90101978068966C05
S11304000E947A0108959C0140E050E06CEF72E490
S113041085E090E00E941103C9010197966C0E9447
S11304207A01089590E087709070986970E0629501
S11304307295707F7627607F76277070862B972B56
S11304400E947A0108959498839BFECF089588ECC6
S113045092E80E947A0181E89AEC0E947A0183E88A
S11304609AEC0E947A010895949881E0839980E03F
S1130470089580E090EB0E947A01089588E092E864
S11304800E947A0108950F931F93CF93DF938C01F9
S1130490C62F88E392E80E947A010E9423028AEA26
S11304A098EB0E947A010E9423028AEA98EB0E9448
S11304B07A010E9423028AEA98EB0E947A010E9440
S11304C023028DE298EB0E947A010E94230284EDBC
S11304D098EB0E947A01CC2399F0C8010196C1508F
S11304E09C012C0F311DE9010E942302F801819126
S11304F08F0190E0986B0E947A010C171D07A1F7F9
S11305000E94230288E092E80E947A01DF91CF9151
S11305101F910F9108950F931F93CF93DF938C0135
S1130520D62F88EC92E80E947A0181E89AEC0E9426
S11305307A0183E89AEC0E947A01DD2399F0C801DC
S11305400196D1509C012D0F311DE9010E94230217
S113055080E090EB0E947A01F80181938F01EC17FF
S1130560FD07A1F788E092E80E947A01DF91CF911C
S11305701F910F9108951F93CF93DF93182FD62FB8
S1130580C42F88E392E80E947A010E9423028AEA37
S113059098EB0E947A010E9423028AEA98EB0E9457
S11305A07A010E9423028AEA98EB0E947A010E944F
S11305B023028DE298EB0E947A010E94230284EDCB
S11305C098EB0E947A010E942302812F90E0986B9D
S11305D00E947A010E9423028D2F90E0986B0E9462
S11305E07A010E9423028C2F90E0986B0E947A017A
S11305F00E94230280E098EB0E947A010E94230269
S113060088E092E80E947A018FEF90E7A2E081509F
S11306109040A040E1F700C00000DF91CF911F910E
S11306200895A1E21A2EAA1BBB1BFD010DC0AA1F2F
S1130630BB1FEE1FFF1FA217B307E407F50720F047
S1130640A21BB30BE40BF50B661F771F881F991FC2
S11306501A9469F760957095809590959B01AC010B
S1130660BD01CF01089597FB092E05260ED057FD35
S113067004D0D7DF0AD0001C38F45095409530954B
S113068021953F4F4F4F5F4F0895F6F79095809512
S1130690709561957F4F8F4F9F4F0895F894FFCFCA
S10506A0020052
S9030000FC
